:10000000012883120313850183168501831286015B
:100010008316860183128701831687018312880164
:1000200083168801831289018316890107309F0096
:100030008312FF3085008600870088008900E83041
:10004000A0000330A1002F208501860187018801CF
:100050008901E830A0000330A1002F2019282008D2
:10006000210403194628A201043022020318412862
:10007000A301B030230203183F28A30A3928A20A9B
:0E0080003428A003200A0319A1032F2808002A
:02400E00323F3F
:00000001FF
